:100000000C941E060C9415280C9442280C94460659
:100010000C94E8120C9446060C9446060C94460682
:100020000C9446060C9446060C9446060C94460620
:100030000C9446060C9446060C9446060C94460610
:100040000C946F280C9446060C94402C0C94832C32
:100050000C9446060C9446060C9446060C944606F0
:100060000C9446060C9446069318F518D418D71825
:10007000DA18DD18E018E318E618F518EF18271A53
:10008000291A291A271A291A291A291A291A291A5A
:10009000291A291A291A291A291A291A291A291A48
:1000A000AD19291A291A291A291A291A1E19291AC1
:1000B000291A291A291A291A291A291A291A291A28
:1000C000291A291A291A291A291A291AB919B919FA
:1000D000B919B919B919B919B919B919B919291A1F
:1000E000291A291A291A291A291A1E19B819B819E8
:1000F000B819B819291AC619CC19D219D819DE1984
:10010000E419EA19F019FA19041A0E1A181A5F19E3
:100110002119291A291A291A291AAD19291A291A4D
:10012000291A291A291A291A291A291AB719B7199D
:10013000B719B719291AC619CC19D219D819DE1945
:10014000E419EA19F019FA19041A0E1A181A5F19A3
:100150002119291A291A291A291AAD195C1A5C1AA7
:100160005C1A5C1A5C1A5C1A5C1A5C1A5C1A5C1ADF
:100170005C1A5C1A5C1A721B721B721B721B721B5C
:10018000721BA11AAB1AB51ABF1A1C1B261B351BF2
:10019000461BCE1CE31CEF1CF81C071D2C1D351D37
:1001A0007E1D471D932099209F20A620B420D62095
:1001B000F420456E746572206D656E752E2E2E00CE
:1001C000546F67676C6564206D6963726F50504D42
:1001D00000546F67676C656420696E76657274653C
:1001E000642050504D2100546F67676C6564205443
:1001F00058206D7574696E672100546F67676C6570
:10020000642074656C656D65747279210050726F3D
:10021000746F636F6C206572726F72207769746897
:100220002052580054696D656F7574207768656E4B
:1002300020636F6E6E656374696E6720746F205201
:100240005800507265737320616E79206B65792058
:10025000746F2063616E63656C00436F6E6E6563DF
:1002600074696E6720746F2052582C20706F776508
:100270007220757020746865205258202877697440
:10028000682062696E6420706C7567206966206EF4
:100290006F74207573696E6720616C776179732064
:1002A00062696E642900546F67676C656420276912
:1002B0006D6D656469617465206F75747075742700
:1002C00000546F67676C65642027736C61766520E6
:1002D0006D6F64652700546F67676C6564202761E4
:1002E0006C776179732062696E642700546F676769
:1002F0006C65642050504D206368616E6E656C20A3
:100300006C696D69740053657420525353492069B8
:100310006E6A656374696F6E206368616E6E656C8A
:100320002028303D3D64697361626C652900536526
:10033000742050504D206D696E696D756D20737914
:100340006E630053657420626561636F6E20696E31
:1003500074657276616C0053657420626561636FC9
:100360006E2064656C617900536574206265616319
:100370006F6E206672657175656E637920696E2097
:10038000487A3A20303D64697361626C652C205074
:10039000783D504D52206368616E6E656C20782CFC
:1003A0002046783D465253206368616E6E656C202E
:1003B00078005365742050574D2073746F7020641B
:1003C000656C61792028302064697361626C6564B2
:1003D0002C20312D323535203D3D20302E317320FB
:1003E0002D2035306D696E29005365742050504DB5
:1003F0002073746F702064656C61792028302064EC
:10040000697361626C65642C20312D323535203D75
:100410003D20302E3173202D2035306D696E29003E
:10042000536574206661696C736166652064656CF0
:1004300061792028302064697361626C65642C20C6
:10044000312D323535203D3D20302E3173202D2089
:1004500035306D696E29002A2A2A2A2A2A2A2A2A50
:100460002A2A2A2A2A2A2A2A2A2A2A2A2A2A2A2AEC
:100470002A2A2A2A0052582041636B6564202D20C5
:1004800072657665727420737563636573736675E0
:100490006C21002A2A2A2A2A2A2A2A2A2A2A2A2AAD
:1004A0002A2A2A2A2A2A2A2A2A2A2A2A2A2A2A2AAC
:1004B000002A2A2A2A2A2A2A2A2A2A2A2A2A2A2AC6
:1004C0002A2A2A2A2A2A2A2A2A2A2A2A2A2A00528E
:1004D000582041636B6564202D20757064617465DC
:1004E000207375636365737366756C21002A2A2A0D
:1004F0002A2A2A2A2A2A2A2A2A2A2A2A2A2A2A2A5C
:100500002A2A2A2A2A2A2A2A2A2A0056616C696457
:100510002063686F69636573206172653A205B319F
:100520005D2D5B31365D20286368616E6E656C20E1
:10053000312D31362900536574206F7574707574D0
:1005400020666F7220706F727420005B585D2061AE
:10055000626F7274206368616E67657320616E6498
:10056000206578697420525820636F6E6669670051
:100570005B535D20736176652073657474696E6783
:100580007320746F205258005B525D20726576654F
:1005900072742052582073657474696E6773207486
:1005A0006F2064656661756C747300557365206EA9
:1005B000756D62657273205B312D445D20746F2010
:1005C0006564697420706F727473205B452D515D92
:1005D00020666F722073657474696E677300202DD6
:1005E00020726563656976657220636F6E66696700
:1005F000757261746F722C20727820737720000AF4
:100600000A6F70656E4C52536E67200053657420FC
:1006100073657269616C2062617564726174653AB8
:10062000200056616C69642063686F696365733A82
:100630002031202D20342B34202F2032202D203823
:10064000202F2033202D20382B34202F2034202D14
:10065000203132202F2035202D2031322B34202FF5
:100660002036202D20313600536574204368616E9A
:100670006E656C20636F6E6669673A20005365741F
:100680002044617461726174652028302D32293AEA
:10069000200053657420486F70206368616E6E653A
:1006A0006C7320286D61782032342C207365706162
:1006B000726174656420627920636F6D6D61732966
:1006C0002076616C69642076616C75657320312DCC
:1006D0003235353A2000536574206368616E6E656B
:1006E0006C2073706163696E6720287831306B48C5
:1006F0007A293A200053657420524620706F77653E
:10070000722028302D37293A200053657420524634
:10071000206D6167696320286865782920652E67E8
:100720002E20307844454144463030443A2000532E
:1007300065742062617365206672657175656E63AC
:10074000792028696E20487A293A20005B5A5D207A
:10075000656E746572207265636569766572206383
:100760006F6E66696775726174696F6E2075746902
:100770006C79005B465D20646973706C61792061FF
:10078000637475616C206672657175656E63696509
:10079000732075736564005B525D2063616C6375E3
:1007A0006C6174652072616E646F6D206B65792079
:1007B000616E6420686F70206C697374005B495DC2
:1007C000207265696E697469616C697A6520736508
:1007D0007474696E677320746F20736B65746368DB
:1007E0002064656661756C7473005B585D2072658A
:1007F00076657274206368616E67657320616E64EC
:100800002065786974206D656E75005B535D20739B
:100810006176652073657474696E677320746F20E8
:10082000454550524F4D20616E64206578697420B3
:100830006D656E7500557365206E756D62657273BA
:10084000205B302D395D20746F20656469742070E1
:100850006172616D657465727300202D2053797328
:1008600074656D20636F6E66696775726174696F18
:100870006E000A0A6F70656E4C52536E672000510D
:1008800029204F7574707574206265666F726520DB
:100890006C696E6B20283D465329203A2000502970
:1008A00020536C617665206D6F64652028657870D3
:1008B0006572696D656E74616C293A20004F29205C
:1008C00054696D65642042494E44206174207374FC
:1008D000617274757020203A20004E292050504DCE
:1008E000206F7574707574206C696D69746564200F
:1008F000202020203A200044495341424C454400E6
:100900004D292050504D205253534920746F20637D
:1009100068616E6E656C202020203A20004C2920F2
:1009200050504D206D696E696D756D2073796E63E1
:10093000202875732920203A200044495341424C15
:100940004544004B29204661696C736166652062ED
:100950006561636F6E20696E74762E2028312D32AA
:10096000353573293A20004A29204661696C736144
:10097000666520626561636F6E2064656C617920D5
:1009800028302D323535203D3E20313073202D204A
:100990003135306D696E293A200049292046616958
:1009A0006C7361666520626561636F6E206672714B
:1009B0002E203A200048292050574D2073746F7024
:1009C0002064656C6179202020202020203A2000BE
:1009D00047292050504D2073746F702064656C61FE
:1009E00079202020202020203A200046292046611E
:1009F000696C736166652064656C617920202020D4
:100A00002020203A200050574D206368616E6E65AB
:100A10006C200066756E6374696F6E3A2000292041
:100A2000706F72742000506F776572546F776572C3
:100A300000445446205548462033322D62697420C4
:100A400031306368004F70656E4C52536E67525878
:100A5000206D696E6920342F36636800466C7974A6
:100A6000726F6E2F4F72616E6765525820554846FF
:100A70002038636800525820747970653A20004429
:100A8000697361626C656400487A00203D3D200016
:100A900043616C63756C61746564207061636B6540
:100AA0007420696E74657276616C3A200042292068
:100AB0004D6963726F202868616C66292050504D23
:100AC000202020203A00412920496E766572746505
:100AD000642050504D20696E20202020203A0030A4
:100AE00029204D7574652062757A7A657220286DAB
:100AF0006F73746C79293A003929205365726961E2
:100B00006C2062617564726174653A00736D617224
:100B100074506F7274004672536B79005472616E38
:100B200073706172656E740044697361626C6564B0
:100B30000038292054656C656D657472793A2020FF
:100B40002020202020003729204368616E6E656CCC
:100B500020636F6E6669673A202000362920446161
:100B60007461726174652028302D32293A2020206A
:100B700000352920486F70206368616E6E656C7364
:100B80003A2020202020003429204368616E6E65C1
:100B90006C2073706163696E673A202000332920EE
:100BA000524620706F7765722028302D37293A2001
:100BB0002020003229205246206D616769633A2067
:100BC0002020202020202020003129204261736530
:100BD000206672657175656E63793A202020000089
:100BE00000000700020100000304060000000000EE
:100BF00000000001020408102040800102040810D7
:100C00002001020408102004040404040404040263
:100C10000202020202030303030303000000002395
:100C2000002600290000000000250028002B0000FD
:100C3000000000240027002A0000F72D11241FBE09
:100C4000CFEFD8E0DEBFCDBF13E0A0E0B1E0ECEF26
:100C5000F1E602C005900D92A83CB107D9F716E065
:100C6000A8ECB3E001C01D92A039B107E1F71CE088
:100C7000CCE3DCE004C02297FE010E94002FCA33BF
:100C8000D107C9F70E94332E0C94FC300C9400005D
:100C900080917505813019F482E08093750580910B
:100CA0007505833019F484E0809375050895A8953F
:100CB0000895DC01ED91FC910190F081E02D099502
:100CC00008952091760530917705382748E0C901CD
:100CD000880F991F37FF06C09C0151E2252750E17C
:100CE000352701C09C01415091F73093770520933F
:100CF0007605089588E38093780580E092ECA1E082
:100D0000B0E08093790590937A05A0937B05B0932A
:100D10007C0587E08093850580E091EAACEBB3E346
:100D200080937D0590937E05A0937F05B093800509
:100D300085E0809386058DEE9EEFADEABEED809353
:100D4000810590938205A0938305B0938405E7E81D
:100D5000F5E080E090E0863028F4DC01AF54BC4F31
:100D60002C9101C020E0219301968831910599F7DB
:100D700082E080939F058AE08093A005089580E03B
:100D80009EECADEEB4E38093BD059093BE05A093B9
:100D9000BF05B093C00580E090E0A0E0B0E580938F
:100DA000C1059093C205A093C305B093C405E5ECBB
:100DB000F5E080E081938F5F8031E1F70895A0E056
:100DC000B0E0E5EEF6E00C94C92ED82F0E94C528BD
:100DD0006115710581059105C9F30E946C2F109270
:100DE0008105109282051092830510928405C4E05B
:100DF000812C912C54018A94C0908105D090820559
:100E0000E0908305F0908405FE2CED2CDC2CCC24A6
:100E10000E94672FA50194010E94A82E6C0D7D1DD4
:100E20008E1D9F1D609381057093820580938305BD
:100E300090938405C15001F7DD2309F450C007E801
:100E400015E0E801A12CB12C62E3C62ED12CE12CD7
:100E5000F12C8881882309F442C0B39419F40E94CC
:100E60007A063DC00E94672FA70196010E94A82E16
:100E7000E1E0E60FA7E8B5E08A2F801B8A1520F491
:100E80008D918E13F9CFE9CF2091860530E0A0E156
:100E9000B7E20E94402E9B01AC01AE2FB0E00E9451
:100EA0004F2E40907D0550907E0560907F0570909C
:100EB0008005640D751D861D971D4090BD055090E1
:100EC000BE056090BF057090C005461657066806BF
:100ED000790618F2E993A39488E1A812BACFCDB7A6
:100EE000DEB7E0E10C94E52E8436910520F4BC01D8
:100EF00080E090E017C09C018E3B910528F42A55B4
:100F00003109AAE0B0E00CC0823D910528F4245BD1
:100F10003109A4E6B0E004C02D5C3109A8E5B2E0D7
:100F20000E94402EA4E6B0E09B01AC010E944F2E2F
:100F3000089590E08C599F4F0E947407089561E0D6
:100F400089E00E94722960E089E00E94AB2908953F
:100F5000892B11F061E001C060E089E00E94AB29BB
:100F6000089560E08EE00E94722961E08FE00E94A7
:100F7000722961E082E00E94722960E083E00E94B1
:100F8000722961E084E00E947229089542E050E0F5
:100F900068E476E081E00E94F5270895E3E0F0E060
:100FA00089E080935700E491E67081E0E63009F033
:100FB00080E00895CF93DF93C82F0E94CE07882347
:100FC00081F0DFB781E080937405F8940E945706A2
:100FD00088E180936000C0936000C1110E945706B1
:100FE000DFBFDF91CF9108958F929F92AF92BF9212
:100FF000CF92DF92EF92FF92CF93FC01C0A5EC2F2E
:10100000E770F0E0E758FC4FA081B0E0C7FF03C0F5
:1010100024E130E002C02FE030E0FC0197A183E141
:10102000989FF0011124E25CFE4F80809180A280A5
:10103000B380A20FB31F20E43FE14DE750E00E94D0
:101040005A2EA50194010E94862E8C2F887149F496
:1010500069017A01E0EDCE0EE7E0DE1EE11CF11C35
:101060001BC0C7FF05C060E47AE88CE29EE004C0C4
:1010700060E07EEE8AEB9BE069017A01F8EBCF0E2F
:10108000FBE0DF1EE11CF11CA50194010E94862EED
:10109000C20ED31EE41EF51EC701B60169517C4F76
:1010A0008F4F9F4F28EE33E040E050E00E94862EA5
:1010B000A8EEB3E00E944F2ECF91FF90EF90DF900B
:1010C000CF90BF90AF909F908F9008958F3F9105E4
:1010D00051F048F0811522E0920738F081159340D5
:1010E00030F482E0089580E0089581E0089583E07F
:1010F0000895A0E0B0E0EFE7F8E00C94D22EEB0109
:101100008A01B82FB695A0E028813981F8012083A3
:101110002A813B8121832C813D8122832E813F8145
:101120002383688179814A815B812C813D81EE81B5
:10113000FF819F2F9295990F990F907C272F2370F5
:10114000922B252F2370220F220F922B232F2370F7
:101150002295207F922BF80194830B5F1F4F2896D6
:10116000AF5FBA1788F680FF24C0888199810E94FA
:101170006608D82E8A819B810E946608E82E8C81A1
:101180009D810E946608F82E8E819F810E946608CC
:10119000F0E4DF9EA001112490E1E99E900111246A
:1011A000242B282BE4E0FE9EB0011124262BF8010D
:1011B0002083CDB7DEB7E7E00C94EE2E803223E03B
:1011C000920708F1883E23E0920740F48F51934044
:1011D000E4E096958795EA95E1F70895803D27E04C
:1011E000920718F48C5D93400895883928E092079F
:1011F00068F4885C974074E0969587957A95E1F756
:101200008D509C4F089580E090E008958FEF93E01B
:1012100008958C30910540F4A4E0880F991FAA9599
:10122000E1F7885D9C4F0895843F23E0920718F40E
:1012300084529C4F0895811524E0920740F486570C
:10124000934FF4E0880F991FFA95E1F7089580E92C
:1012500098E008959C013695279525753575821B74
:10126000930B9C0123733373969587959695879579
:1012700083739373820F931F9C0154E036952795D7
:101280005A95E1F7280F391F2F703F7041E051E068
:10129000249FC001259F900D349F900D1124892F0C
:1012A00008955A98882319F00000419A02C000005E
:1012B000419800005A9A000008955A9A000086B199
:1012C0005A98000081700895CF93DF93D82F5C9ACD
:1012D0005A985C98C8E08D2F80780E945109DD0FE4
:1012E000C150C9F75A98DF91CF9108958F770E9426
:1012F00064090895CF93DF93D82FC8E08D2F8078AD
:101300000E945109DD0FC150C9F75A98DF91CF9162
:101310000895CF93DF935A98C8E080E0D82FDD0F6F
:101320000E945D098D0FC150C9F7DF91CF910895DB
:101330000E9476090E9489095C9A0895A1E0B0E0B4
:10134000E4EAF9E00C94D72E806869830E9464096E
:101350006981862F0E947A095C9A2196E2E00C94BA
:10136000F32ECF93C0918105C827E82FF0E0E8580D
:10137000FA4F678589E70E949E096C2F8DE30E94D2
:101380009E096C2F82E40E949E09CF91089586E207
:101390000E9498090895CF93DF93EC016C818CE152
:1013A0000E949E096D818DE10E949E096E818EE1F1
:1013B0000E949E096F8180E20E949E09688581E2F9
:1013C0000E949E09698582E20E949E096A8583E2E5
:1013D0000E949E096B8584E20E949E096C8585E2CD
:1013E0000E949E096D858AE20E949E096E858EE6A6
:1013F0000E949E096F858FE60E949E09688980E79A
:101400000E949E09698981E70E949E096A8982E794
:101410000E949E09DF91CF910895CF92DF92EF92C3
:10142000FF92CF93DF936B017C01C11488E3D80650
:101430008CE9E8068CE1F80628F5C701B60120E83A
:1014400036E948E950E00E94862EE901689760E895
:1014500079E687E69FEF0E94622E6C0D7D1D8E1D42
:101460009F1DF2E0660F771F881F991FFA95D1F72D
:1014700021E732E040E050E00E94862EF22EE32E7B
:1014800080E421C0C701B60120E03DE241E351E024
:101490000E94862EE901689760E073ED8EEC9EEF66
:1014A0000E94622E6C0D7D1D8E1D9F1D660F771F85
:1014B000881F991F21E732E040E050E00E94862E0D
:1014C000F22EE32E80E66C2F6F71680F85E70E9485
:1014D0009E096E2D86E70E949E096F2D87E70E9468
:1014E0009E09DF91CF91FF90EF90DF90CF9008950C
:1014F000682F8DE60E949E0908958F929F92AF9269
:10150000BF92CF92DF92EF92FF92CF93DF93D82FCB
:1015100083E00E9498098093730584E00E949809F3
:101520008093720560E086E00E949E0961E087E09A
:101530000E949E096FE789E00E949E0965E08AE0AB
:101540000E949E0962E18BE00E949E0965E18CE0A9
:101550000E949E096DEF8DE00E949E0960E08EE082
:101560000E949E09DD2319F08BE291E008C02091D2
:101570009F0533E1239FC0011124825C9E4F0E948E
:10158000CB096CE880E30E949E096FE082E30E9431
:101590009E0962E483E30E949E098091A00587FF73
:1015A00002C064E101C06AE084E30E949E096AE22D
:1015B00085E30E949E096DE286E30E949E0964ED28
:1015C00087E30E949E0960E088E30E949E0960E034
:1015D00089E30E949E09D11109C0C0908105D09075
:1015E0008205E0908305F090840507C0C5E9CC2E04
:1015F000C1ECDC2EED2CCEEDFC2ECAE38F2C992411
:10160000AA24BB24682D8C2F0E949E09682D85E09A
:101610008C0F0E949E09FE2CED2CDC2CCC24CF5F7D
:10162000CE3361F76FEF83E40E949E096FEF84E48D
:101630000E949E096FEF85E40E949E096FEF86E489
:101640000E949E09DD2311F066E002C060918505CD
:101650008DE60E949E0960E089E70E949E096091E4
:1016600086058AE70E949E0960E083E70E949E0942
:1016700060E084E70E949E09D11109C060917D0558
:1016800070917E0580917F059091800504C060E097
:1016900071EA8CEB93E30E940D0ADF91CF91FF90EA
:1016A000EF90DF90CF90BF90AF909F908F90089574
:1016B00061E087E00E949E0964E28EE70E949E0935
:1016C00063E088E00E949E0960E088E00E949E0935
:1016D00065E087E00E949E0962E085E00E949E0925
:1016E00083E00E9498098093730584E00E94980922
:1016F00080937205089583E00E9498098093730592
:1017000084E00E9498098093720561E087E00E945E
:101710009E096AE070E080E090E00E94E8280E9464
:10172000580B00000895CF92DF92FF920F931F9302
:10173000CF93DF931F92CDB7DEB7082F162F8EE31E
:1017400099830E949E09F02EC02E9981D92E8C2D4E
:101750008F19811738F4F60161916F018FE70E94AC
:101760009E09F5CF64E085E00E949E0983E00E9417
:1017700098098093730584E00E949809809372050C
:101780000E94C52860936E0570936F058093700565
:101790009093710569E087E00E949E0981E0809343
:1017A00075050F90DF91CF911F910F91FF90DF9002
:1017B000CF9008950F931F930E94930B809175050E
:1017C000813099F40E94C52800916E0510916F0533
:1017D0002091700530917105601B710B820B930B8A
:1017E000603A76488140910548F3809175058130D3
:1017F00031F46DE971E084EE95E00E94942A1F9126
:101800000F9108950F931F9380917505823021F4F5
:101810001092750581E020C0809175058130D9F462
:101820000E94C52800916E0510916F0520917005EA
:1018300030917105601B710B820B930B613A7648F6
:101840008140910540F061E087E00E949E0910927E
:10185000750582E001C080E01F910F910895CF933C
:10186000DF93EC014AE050E06D2F70E084EE95E0EC
:101870000E94622B6EE284EE95E00E94662ABE0111
:1018800084E0769567958A95E1F76F7077274AE04F
:1018900050E084EE95E00E94622B6EE284EE95E0CB
:1018A0000E94662ABE016F7077274AE050E084EEFE
:1018B00095E00E94622BDF91CF910895D82FC0E070
:1018C000CD1780F42C9A64E670E080E090E00E94EE
:1018D000E8282C9864E670E080E090E00E94E82818
:1018E000CF5FEECF6CE271E080E090E00E94E828EC
:1018F000E6CF0F931F93CF93DF93EC01062F15E0F4
:10190000115051F0CE010E94E330081741F0602FD2
:10191000CE010E94EB30F4CF82E00E945E0CDF919A
:10192000CF911F910F910895A0E0B0E0EAE9FCE0AB
:101930000C94C92E482E562EC0E0D0E0612C712C9C
:10194000E12CF12C00E010E041100CC06090D605B5
:1019500086E4689E3001112459E1E52EF12C0CEB50
:1019600015E01EC091E049120FC06090D605E6E474
:101970006E9E30011124FBE16F0E711C49E2E42ED2
:10198000F12C08E715E00CC082E0481209C028E1FC
:10199000622E77247394EE24E394F12C05ED15E088
:1019A00043018C0E9D1E109277051092760534012E
:1019B000A62CA818B12CC30101966C01AE14BF046B
:1019C000A8F4A00EB11E511006C0C3010E94E3305E
:1019D000F501808305C0F5016081C3010E94790C87
:1019E000F50180810E9461063601E2CFC3015110EA
:1019F00018C0C3010E94E330B82EC6010E94E33034
:101A00002B2D30E0322F2227282B809176059091C4
:101A100077058217930779F4C0E0D0E055245394FA
:101A200093CF3601609177050E94790C609176051D
:101A3000C6010E94790CC05EDE4FC13E92E0D9071C
:101A400008F482CF852DCDB7DEB7E0E10C94E52E0A
:101A500061E082E00E94940C089560E082E00E94C0
:101A6000940C8091D505853020F01092D5050E9408
:101A7000280D8091D5058093D605089561E080E01A
:101A80000E94940C61E081E00E94940C089560E053
:101A900080E00E94940C882351F060E081E00E9475
:101AA000940C882321F080917805883349F00E94B6
:101AB000BF060E947A0681E00E94DF060E943E0D6A
:101AC0000895882319F069EA71E002C06DEA71E0B7
:101AD00084EE95E00E94942A0895FF920F931F933D
:101AE000CF93DF9369EC7BE084EE95E00E94402A7F
:101AF00040917D0550917E0560917F057091800534
:101B00002AE030E084EE95E00E94692B63EB7BE0F5
:101B100084EE95E00E94402A409181055091820513
:101B2000609183057091840520E130E084EE95E0BA
:101B30000E94692B6DE97BE084EE95E00E94402ACB
:101B40004AE050E06091850584EE95E00E94912B7B
:101B500067E87BE084EE95E00E94402A4AE050E08E
:101B60006091860584EE95E00E94912B61E77BE011
:101B700084EE95E00E94402AC7E8D5E0F12C8E0162
:101B800088818823A9F0FF2031F060EB71E084EEBA
:101B900095E00E94632A21964AE050E0F8016081B6
:101BA00084EE95E00E945A2BF394F8E1FF12E7CF00
:101BB00084EE95E00E946E2A6BE57BE084EE95E072
:101BC0000E94402A4AE050E060919F0584EE95E033
:101BD0000E94912B66E47BE084EE95E00E94402A0F
:101BE000E091A005E770F0E0EE0FFF1FEF57FC4F0C
:101BF0006081718184EE95E00E94942A61E37BE02C
:101C000084EE95E00E94402A8091A005887188307A
:101C100069F028F4811113C068E27BE00CC08031C8
:101C200041F0883161F46CE07BE005C06CE17BE061
:101C300002C066E17BE084EE95E00E94822A68EFB4
:101C40007AE084EE95E00E94402A40917905509117
:101C50007A0560917B0570917C052AE030E084EE86
:101C600095E00E94692B6FED7AE084EE95E00E948A
:101C7000402A8091C10580710E94610D66EC7AE076
:101C800084EE95E00E94402A8091C10580740E94F4
:101C9000610D6DEA7AE084EE95E00E94402A809121
:101CA000C10580720E94610D60E97AE084EE95E0E2
:101CB0000E94402A88E795E00E94F407AB01BC012E
:101CC0002AE030E084EE95E00E944B2B6BE87AE04E
:101CD00084EE95E00E94402A88E795E00E94F40790
:101CE0009B01AC0160E472E48FE090E00E94862EDC
:101CF000BA01A9012AE030E084EE95E00E944B2B66
:101D000068E87AE084EE95E00E94822ACDB7DEB7DB
:101D1000E5E00C94F02E8F929F92AF92BF92CF92FB
:101D2000DF92EF92FF92811107C06FE77AE084EEB5
:101D300095E00E94822A2FC090E00E94740724E65A
:101D400030E040E050E00E94862ECA01B9012AE04E
:101D500030E040E050E00E94862E49015A016B01BC
:101D60007C012AE030E0B501A40184EE95E00E94F8
:101D70004B2B6EE284EE95E00E94662A2AE030E06A
:101D8000B701A60184EE95E00E944B2B63E784EE39
:101D900095E00E94A62AFF90EF90DF90CF90BF9031
:101DA000AF909F908F9008951F93CF93DF9365E737
:101DB0007AE084EE95E00E94402A8091A10581306E
:101DC00041F46CE57AE084EE95E00E94822A10E00E
:101DD00050C0823019F465E47AE0F5CF843019F40C
:101DE00061E37AE0F0CF853091F766E27AE0EBCFFD
:101DF000C12FD0E0C930D1050CF441C068E3610FB8
:101E000084EE95E00E94662A6EE17AE084EE95E029
:101E10000E94402ABE016F5F7F4F4AE050E084EE8F
:101E200095E00E942A2B63E17AE084EE95E00E941F
:101E3000402ACF55DA4FE981E03218F566E07AE0C2
:101E400084EE95E00E94402A8981803130F06CE672
:101E500073E084EE95E00E94632A69816F7070E000
:101E60006F5F7F4F4AE050E084EE95E00E94332B95
:101E70001F5F80914A05181708F4BACF0FC061E3BD
:101E8000BECFEF70F0E0EE0FFF1FEF56FC4F60810A
:101E9000718184EE95E00E94942AEACF6BEE79E09E
:101EA00084EE95E00E94402A8091B9050E948B0E35
:101EB00060ED79E084EE95E00E94402A8091BA05B9
:101EC0000E948B0E65EB79E084EE95E00E94402A3B
:101ED0008091BB050E948B0E6AE979E084EE95E063
:101EE0000E94402A4091B1055091B2056091B3051E
:101EF0007091B405411551056105710539F12AE06C
:101F000030E084EE95E00E94692B67E679E084EE8C
:101F100095E00E94402A8091B5050E949907AB0187
:101F2000BC012AE030E084EE95E00E94692B63E476
:101F300079E084EE95E00E94402A4AE050E060910A
:101F4000B60584EE95E00E94912B06C06AE379E025
:101F500084EE95E00E94822A6DE179E084EE95E0BE
:101F60000E94402A6091B7057091B8054AE050E0A0
:101F700084EE95E00E947B2B60E079E084EE95E0B2
:101F80000E94402A6091B005603450F470E06F5FA9
:101F90007F4F4AE050E084EE95E00E94332B06C06C
:101FA00067EF78E084EE95E00E94822A6AED78E09F
:101FB00084EE95E00E94402A8091AF0580FF03C027
:101FC00062EB71E002C066EB71E084EE95E00E9486
:101FD000942A6DEB78E084EE95E00E94402A80918F
:101FE000AF0582700E94610D6EE978E084EE95E0A5
:101FF0000E94402A8091AF0584700E94610D6FE7B6
:1020000078E084EE95E00E94402A8091AF058870C8
:102010000E94610DDF91CF911F9108950F931F933F
:10202000CF93DF93209147052F3FA9F56FEF75E020
:1020300084EE95E00E94402A88E893E00E942F0CED
:102040006EED75E084EE95E00E94402A809148058F
:10205000909149050E942F0C6BEA75E084EE95E0A3
:102060000E94822A68E875E084EE95E00E94822A48
:1020700060E775E084EE95E00E94822A6BE475E0EB
:1020800084EE95E00E94822A84EE95E00E946E2AFA
:102090000E94D40E68C012160CF065C0332727FDCD
:1020A000309580914A0590E0821793070CF45BC04D
:1020B00066E375E084EE95E00E94402A6091470552
:1020C000772767FD70954AE050E084EE95E00E9426
:1020D000332B6BE075E084EE95E00E94402A10E01F
:1020E00008E280914B051817D0F5C12FD0E0CC0F36
:1020F000DD1FC45BDA4F288130E0809147059927C6
:1021000087FD909501972817390739F56AEB71E03B
:1021100084EE95E00E94632A4AE050E0602F84EE4E
:1021200095E00E945A2B6EEB71E084EE95E00E94E0
:10213000632AE981EF70F0E0EE0FFF1FEF56FC4FCE
:102140006081718184EE95E00E94632A62EC71E007
:1021500084EE95E00E94632A0F5F1F5FC2CF84EE7A
:1021600095E00E946E2ADF91CF911F910F91089503
:10217000FF920F931F93CF93DF93C7E8D5E0F12C25
:102180008E0188818823D1F164EC71E084EE95E0C2
:102190000E94632A4AE050E06F2D84EE95E00E9491
:1021A0005A2B61ED71E084EE95E00E94632A21963E
:1021B000F801208130E0A0E1B7E20E94402E9B01AF
:1021C000AC01A0918605B0E00E944F2EAB01BC018E
:1021D00080917D0590917E05A0917F05B09180054D
:1021E000480F591F6A1F7B1F2AE030E084EE95E0FC
:1021F0000E94692BF394F8E1FF12C2CFCDB7DEB78E
:10220000E5E00C94F02E1092E10485E6E2EEF4E0B5
:10221000DF011D928A95E9F70895CF93C82F8F3774
:1022200019F0883009F045C0E091E104EE23D9F1BE
:10223000E150E093E104F0E0EE51FB4F10826DE0DD
:1022400070E084EE95E00E945906C0E08091E104C0
:10225000C81760F4EC2FF0E0EE51FB4F608170E0A6
:1022600084EE95E00E945906CF5FF0CF60E270E007
:1022700084EE95E00E9459066DE070E084EE95E0F2
:102280000E945906C0E08091E104C81778F5EC2F50
:10229000F0E0EE51FB4F608170E084EE95E00E942B
:1022A0005906CF5FF0CF67E084EE95E00E94662A82
:1022B0001DC08B3119F40E9403111AC08D30C1F07A
:1022C0008A30B1F08091E104843668F76C2F70E0B9
:1022D00084EE95E00E945906E091E10481E08E0FC2
:1022E0008093E104F0E0EE51FB4FC08380E001C039
:1022F00081E0CF910895CF93C82F0E94C5286093A5
:10230000CA047093CB048093CC049093CD04C09303
:10231000DF04CC2329F040E051EE60E070E004C01F
:1023200040E855E260E070E084EE95E00E94F02C19
:10233000CF9108959091CE04492F4F7050E0BA018B
:102340006F5F7F4F292F30E0E4E035952795EA95C0
:10235000E1F76217730759F0FA01E153FB4F8083ED
:1023600081E0890F8F70907F892B8093CE04089530
:102370006EE770E084EE95E00E9459060895A3E1AF
:10238000B1E0E5ECF1E10C94CA2EE7E8F5E0712C40
:102390008191882321F0739428E17212F9CF65EDC1
:1023A00071E084EE95E00E94942A4AE050E0672DA7
:1023B00084EE95E00E94912B80E00E947D0A0E94AD
:1023C000580B8E010E5F1F4FC12CD12C7601C39488
:1023D00066246A945C2C0E94B9284B015C01209110
:1023E000860530E0A0E1B7E20E94402E9B01AC01DF
:1023F000C701B6010E94622E20917D0530917E05B5
:1024000040917F0550918005620F731F841F951FB7
:102410002091BD053091BE054091BF055091C0058A
:10242000261737074807590718F4F801608225C0B6
:102430008C2D0E94B10961E070E080E090E00E9484
:10244000E828F80110820E94B928681979098A09D8
:102450009B09643F71408105910540F40E94C709C2
:10246000F8019081981778F78083EDCF50FE03C074
:102470002B982C9A02C02B9A2C982FEFC21AD20AB2
:10248000E20AF20A0F5F1F4F8FEFC816D104E10472
:10249000F10409F09FCFCE019395FC01D82E7FEF78
:1024A00068EC2E2F281B271510F051E056C0DE01D6
:1024B000129651E02FEF41E03D91321710F0322F8C
:1024C00001C0452F5F5F5F3F11F0232FF5CF419390
:1024D000242F30E0A1E0B0E0AC0FBD1FA20FB31F6E
:1024E0005C93413079F0DE01A20FB31F5C93423060
:1024F00049F0AFEFBFEFAC0FBD1FA20FB31F6C933E
:102500004E3F78F6A2E0B0E0AC0FBD1FA20FB31FA4
:102510007C934D3F30F6A3E0B0E0AC0FBD1FA20F9F
:10252000B31F6C93BECF452F242F30E0FC01E20F88
:10253000F31F6081AFEFB0E0AC0FBD1FA20FB31F60
:102540002C91621748F44150DC01A40FB11D2C916D
:1025500020836C934111E8CF5F5F571520F3372D2F
:10256000369520E0231770F4DC01A20FB11D4C91C9
:10257000522F530FFC01E50FF11D50815C934083F6
:102580002E5FF0CFF7E8EF2EF5E0FF2E8C01802FC5
:102590008D19871598F4F801C1908F014AE050E039
:1025A0006C2D84EE95E00E945A2B6CE284EE95E04F
:1025B0000E94662AF701C1927F01E9CF84EE95E07F
:1025C0000E946E2A81E0CD5EDE4FEFE00C94E62E95
:1025D0001F920F920FB60F9211240F931F932F93F8
:1025E0003F934F935F936F937F938F939F93AF939B
:1025F000BF93EF93FF934091C1055091C205609145
:10260000C3057091C40586B18A019B01007411272E
:102610002227332785FB882780F990E0A0E0B0E0EF
:10262000081719072A073B0709F468C0809184003E
:102630009091850010928500109284002091A7044B
:1026400021115CC045FD02C096958795853C29E027
:102650009207C0F180910A0190E0A0E0B0E00CE1A7
:1026600076956795579547950A95D1F74115510588
:102670006105710521F441E050E060E070E0481729
:1026800059076A077B07D8F480910A018F3FB9F098
:1026900040E080910A01481780F4842F90E0880F71
:1026A000991FFC01E957FB4F20813181FC01E55F57
:1026B000FE4F318320834F5FECCF1092A80410921D
:1026C0000A011CC08D3B22E09207A8F020910A016C
:1026D000203188F410910A0121E0210F20930A0192
:1026E0000E94DE08E12FF0E0EE0FFF1FE957FB4FDD
:1026F0009183808303C08FEF80930A01FF91EF9154
:10270000BF91AF919F918F917F916F915F914F9109
:102710003F912F911F910F910F900FBE0F901F901F
:10272000189583E0809380008AE1809381008FEF89
:102730009FEF909389008093880010926F0080E251
:1027400080936C00E8E6F0E08081826080830895E9
:102750000E942D0D8091D605843011F41092D6057B
:1027600008956F3018F086958058089589E0689F25
:10277000802D11240895A0E0B0E0E1ECF3E10C9489
:10278000D12EC82F0E94C528009138041091390419
:1027900020913A0430913B046B017C01C01AD10AAC
:1027A000E20AF30A9701860149E8C41643E1D40618
:1027B000E104F10410F010923C046093380470932B
:1027C000390480933A0490933B042091A7048FEF3F
:1027D000820F8230E8F5E0913C04EE2309F46EC1EB
:1027E000E13011F482E0D8C1E03178F581E08E0F5C
:1027F00080933C04F0E0E957FB4FC083803109F03F
:10280000D4C1E9E8F4E0213029F4A181A695A69588
:10281000808108C080819181A92FA695A695A69553
:1028200096958795A03148F4B0E090E0AA0FBB1FC1
:10283000A55FBE4F11969C938E931092A80432967A
:1028400084E0E739F807F9F6B0C110923C04ADC155
:10285000233009F023C1E0913C04E11118C0CF30CE
:1028600009F011C10E94B9280091B5041091B60475
:102870002091B7043091B804601B710B820B930B4D
:10288000623071058105910508F089C1FCC0E8310D
:1028900048F481E08E0F80933C04F0E0EA57FB4F50
:1028A000C083F1C0E83109F0ECC0C111EAC040E0DA
:1028B00050E0ABE0CA01B3E0880F991FBA95E1F789
:1028C000A49F9001A59F300D1124F901E957FB4FFA
:1028D0006081E1817E2F777075956795FC01EE0F21
:1028E000FF1FE55FFE4F71836083F901E857FB4FDF
:1028F000B081B695B695B695E181FE2FF295FF0FA2
:10290000F07E6F2F6B2BE695E695E6957E2F777020
:1029100075956795FC01EE0FFF1FE35FFE4F718316
:102920006083F901E757FB4FB081B295B695B69534
:10293000B370C181DC2FDD0FDD0F6D2F6B2BC295C6
:10294000C695C695C370E281E170EE0FEE0F7E2F43
:102950007C2B75956795FC01EE0FFF1FE15FFE4F25
:1029600071836083F901E557FB4FB081B695E18132
:10297000FE2FF795FF27F7956F2F6B2BE6957E2F90
:10298000777075956795FC01EE0FFF1FEF5EFE4FA8
:1029900071836083F901E457FB4FB081B295BF703A
:1029A000E181FE2FF295F07F6F2F6B2BE295EF7098
:1029B0007E2F777075956795FC01EE0FFF1FED5E1A
:1029C000FE4F71836083F901E357FB4FB081BB1F5A
:1029D000BB27BB1FC181DC2FDD0F6D2F6B2BCC1FE5
:1029E000CC27CC1FE281E370EE0F7E2F7C2B7595F8
:1029F0006795FC01EE0FFF1FEB5EFE4F7183608356
:102A0000F901E157FB4FB081B695B695E181FE2FF4
:102A1000F295FF0FFF0FF07C6F2F6B2BE695E6957D
:102A20007E2F777075956795FC01EE0FFF1FE95EAD
:102A3000FE4F71836083F901E057FB4F208122959F
:102A4000269527703181E32FEE0FEE0FEE0F6E2FDC
:102A5000622B732F72957695777075956795FC014B
:102A6000EE0FFF1FE75EFE4F718360834F5F5F4F86
:102A70004230510509F01ECF80919D0483FF1092D2
:102A8000A80410923C040E94B9286093B504709386
:102A9000B6048093B7049093B80487C0243009F03B
:102AA00084C060913C0461110BC0C83AB1F410922B
:102AB00077051092760588EA0E94610681E06CC075
:102AC000613019F4C093370404C0623031F4C0930C
:102AD00036048C2F0E9461065AC0E09136042E2FD6
:102AE00030E0220F331F462F50E0C90102968417B1
:102AF00095073CF0633268F7FA01EC57FB4FC0834F
:102B0000E8CF2D5F3F4F8C2F90E06091760570915C
:102B100077054217530749F4982F88278627972768
:102B2000909377058093760532C06817790769F529
:102B300080913704813049F5E13118F080E18093CC
:102B40003604F0903604C8E8D4E000E010E00F1539
:102B5000D0F4FE013197808190E0982F882728815A
:102B6000822B43E0969587954A95E1F70E94DE080F
:102B7000F801EE0FFF1FE55FFE4F918380830F5F2B
:102B80001F4F2296E4CF1092A80410923C0480912B
:102B90003C04882351F08F5F80933C0406C08091F1
:102BA0003C048F5F80933C046ECFCDB7DEB7E8E086
:102BB0000C94ED2EE82FF0E0E454FA4FE185E0317B
:102BC00050F4F894F0E0EE0FFF1FE55FFE4F8081B8
:102BD0009181789408958EE08E0F8B3058F4F0E058
:102BE000E25FF10924E62E9FC0012F9F900D112472
:102BF0000C960895E13F59F018F4E03F89F004C0C5
:102C0000ED3F41F0EE3F49F080E092E0089586E02C
:102C100090E008958AEF93E008958FEF93E0089590
:102C200080E090E00895A2E2B0E0E9E1F6E10C94E2
:102C3000C72E9E012F5F3F4F80E1D9011D928A95DB
:102C4000E9F763E072E084EE95E029A33AA30E94DD
:102C5000942A0E947B0B1D8A1E8A1F8A188E312C93
:102C6000212C00E0812C912C5401412C74E7572E2B
:102C70007BE8672E72E3772EE0E5CE2EE3ECDE2EC6
:102C8000E12CF12C84EF91E0A0E0B0E08D8F9E8FDD
:102C9000AF8FB8A380E09EECADEEB4E3898F9A8F3E
:102CA000AB8FBC8F80E094E7ABE8B2E3898B9A8B63
:102CB000AB8BBC8B84EE95E00E94A82B892B09F48A
:102CC000E1C084EE95E00E94D52B9C0133272C3285
:102CD000310509F442C0ACF42332310509F0ABC030
:102CE00019821A821B821C821D821E821F821886F4
:102CF00019861A861B861C861D861E861F86188AC4
:102D000060C02434310529F02335310509F4B2C0FF
:102D100092C064E484EE95E00E94662A2AE030E0E6
:102D200040E054E76BE872E384EE95E00E94F42AF9
:102D30006CE284EE95E00E94662A2AE030E040E0F2
:102D40005EEC6DEE74E384EE95E00E94F42A6CE292
:102D500084EE95E00E94A62AADCF0F5F043009F003
:102D6000A9CF29813A814B815C81A8EEB3E00E9412
:102D70004F2E698B7A8B8B8B9C8B2D813E814F8163
:102D800058850E944F2E698F7A8F8B8F9C8F298553
:102D90003A854B855C852D8F3E8F4F8F58A32D85AF
:102DA0003E854F8558890E944F2E6B017C01603211
:102DB0003EE473078105910530F462E38CE10E94E3
:102DC0009E0900E077CF603345E7740781059105E0
:102DD00010F462E2F3CF60345CE975078105910578
:102DE00010F466E2EBCF80E5C81683ECD806E10468
:102DF000F10410F462E1E2CF90E6C9169AEED9062A
:102E0000E104F10410F465E1D9CFA0E7CA16A1E10D
:102E1000DA06A1E0EA06F10410F461E0CFCFB0EAEF
:102E2000CB16B6E8DB06B1E0EB06F10410F463E084
:102E3000C5CF65E0C3CF10ED180F1A3008F03ACFB8
:102E4000E1E0F0E0EC0FFD1F24E0029FE00DF11D3A
:102E500011242081318142815381AAE0B0E00E9497
:102E60004F2E610F711D811D911D608371838283BF
:102E7000938320CF49885A886B887C88812C912C39
:102E8000540118CF81149104A104B10489F4C30141
:102E9000B2010E940D0A61E070E080E090E00E94C3
:102EA000E8281D8A1E8A1F8A188E312C22242A9413
:102EB0008D8D9E8DAF8DB8A188169906AA06BB068A
:102EC000D0F40E94C7092D893E894F89588D280F5B
:102ED000311D411D511D2D8B3E8B4F8B588F381648
:102EE00008F4382E821508F4282E3FEF831A930A2F
:102EF000A30AB30A56C0C301B20128EE33E040E092
:102F000050E00E94862EBA01A9012AE030E084EE4A
:102F100095E00E944B2B6CE284EE95E00E94662ABD
:102F20004AE050E0632D84EE95E00E945A2B6CE25B
:102F300084EE95E00E94662A6D897E898F89988D3E
:102F4000A50194010E94862EBA01A9012AE030E071
:102F500084EE95E00E944B2B6CE284EE95E00E949B
:102F6000662A4AE050E0622D84EE95E00E945A2BDA
:102F70006CE284EE95E00E94A62A4C0C5D1C6E1C4F
:102F80007F1C898D9A8DAB8DBC8D84159505A6050A
:102F9000B70520F449885A886B887C88812C912C4D
:102FA000540129893A894B895C89283E334041057F
:102FB000510509F07FCEA296E2E10C94E32EACE13C
:102FC000B0E0E5EEF7E10C94D12E0E94C5286B012C
:102FD0007C0181E00E947D0A14E703E0198361E02F
:102FE000CE0101960E94DA0B009375050E94580BE2
:102FF0006AEF70E080E090E00E94E828809175051B
:10300000833089F484EE95E00E94A82B892B59F433
:103010000E94C5286C197D098E099F096038734C80
:10302000894C9140D8F280917505833009F44FC0E6
:103030008FE70E9476090E9489098983843511F0FF
:1030400083E05CC00E94890910924805809349057D
:103050000E9489092091480530914905280F311DAA
:1030600030934905209348050E94890980934A05B9
:103070000E94890980934B05813110F7F12C0F2DA7
:1030800010E080914B0590E0880F991F08171907F1
:1030900040F40E948909F801E45BFA4F8083F394BD
:1030A000EECF80E7898361E0CE0101960E94DA0BC2
:1030B00083E0809375050E94580B62E370E080E026
:1030C00090E00E94E82880917505833011F482E039
:1030D00015C08FE70E9476090E948909898380358F
:1030E00009F0AECF01EA15E00E948909F801819349
:1030F0008F01F5E00C3B1F07B9F781E06C96E8E023
:103100000C94ED2E80914705992787FD9095A92F66
:10311000B92FFC013196EB30F10508F066C0EC5C8C
:10312000FF4F0C94FE2E62E778E084EE95E00E945B
:10313000822A88E893E00E942F0C6AE578E084EE0A
:1031400095E00E94822A65E378E084EE95E00E9493
:10315000822A6BE078E084EE95E00E94822A6AEE93
:1031600077E084EE95E00E94822A6DEB77E084EEB2
:1031700095E00E94822A67E977E084EE95E00E945C
:10318000822A63E777E084EE95E00E94822A6CE46D
:1031900077E084EE95E00E94822A84EE95E00E941A
:1031A0006E2A0E946D0D21C06FE277E01AC06AE0BE
:1031B00077E017C065EF76E014C066ED76E011C0E9
:1031C00062E976E00EC06DE776E00BC068E676E077
:1031D00084EE95E00E94822A62E276E002C06CE012
:1031E00076E084EE95E00E94822A6AE070E080E05A
:1031F00090E00E94E82884EE95E00E94A82B892B9D
:1032000029F084EE95E00E94D52BF5CF0895ACE12E
:10321000B0E0EDE0F9E10C94D12E909147059F3F8D
:1032200009F023C1482F50E0FA013A97EF36F10533
:1032300008F00FC1E15CFF4F0C94FE2E60E172E0DC
:10324000A0C06CE172E084EE95E00E94942A85E7CC
:1032500089838BE1E1EAF5E0DE01129601900D929F
:103260008A95E1F76CE1CE0101960E94DA0B0E948B
:10327000580B83E08093750568EC70E080E090E087
:103280000E94E82880917505843009F0E2C08FE73C
:103290000E9476090E9489098983853509F0D9C081
:1032A0006DEE74E084EE95E00E94822A6FEC74E08B
:1032B00084EE95E00E94822A61EB74E096C064E39C
:1032C00072E084EE95E00E94942A89E6898361E0A9
:1032D000CE0101960E94DA0B0E94580B83E0809386
:1032E000750568EC70E080E090E00E94E82880912D
:1032F0007505843009F0ADC08FE70E9476090E9401
:10330000890989838E010E5F1F4F7E014DE1E40E16
:10331000F11C0E948909F80181938F01EE15FF05C8
:10332000C1F78BE1FE013296A1EAB5E001900D9262
:103330008A95E1F78981893409F08BC063E974E0EB
:1033400084EE95E00E94822A65E774E084EE95E0C1
:103350000E94822A67E574E048C06EE472E084EE61
:1033600095E00E94942A8EEF8093470572C08052A8
:103370008750805390914A05981708F066C06DE514
:1033800072E084EE95E00E94942A63C084E1809309
:10339000470560E274E029C085E18093470569EE46
:1033A00073E023C086E18093470562EB73E01DC0A4
:1033B00087E18093470568E673E017C088E1809352
:1033C000470567E573E011C089E18093470563E431
:1033D00073E00BC08AE1809347056EE273E005C09D
:1033E0008BE18093470566E073E084EE95E00E94F0
:1033F000822A2FC06CEE72E084EE95E00E94822A51
:103400008091AF0591E01DC066ED72E084EE95E01D
:103410000E94822A8091AF0592E013C061EC72E0B5
:1034200084EE95E00E94822A8091AF0594E009C065
:1034300066EA72E084EE95E00E94822A8091AF05F0
:1034400098E089278093AF058FEF809347050E940E
:103450000E1084EE95E00E94A82B892B09F45AC126
:1034600084EE95E00E94D52BF4CF0E940D118823A5
:1034700009F450C18091E104811104C08FEF809361
:10348000470540C140E050E060E070E082EE94E02B
:103490000E94752F40914705042F112707FD1095B5
:1034A000212F312FF8013197EB31F10508F01AC1C6
:1034B000E255FF4F0C94FE2E552747FD5095209165
:1034C0004A0530E0241735070CF40CC18B019C0130
:1034D0000150110921093109003211052105310579
:1034E00058F0C0904B05EDE4F5E0F12CD12CA8E2AA
:1034F000EA2E415051090FC0FA01EF55FA4F6150C1
:103500006083D8C0DF0111972C9130E02417350774
:1035100029F0F3943296FC10F5CFCAC00E2D10E0BE
:1035200020E030E0061717072807390741F420810B
:10353000DA01AF55BA4F11962C93DD24D394E3945E
:10354000E8CF6F3F71058105910511F008F0CAC001
:103550006093B905AFC06F3F71058105910511F00A
:1035600008F0C0C06093BA05A5C06F3F7105810522
:10357000910511F008F0B6C06093BB059BC0209187
:10358000E20420622037E9F440E050E060E070E0BF
:1035900083EE94E00E94752F9B01AC01DC01CB010E
:1035A0000197A109B1090897A105B10508F0ADC0BF
:1035B000A4EDB0E30E944F2E6A5E7C4A8A46954E87
:1035C00024C02636E9F440E050E060E070E083EE8D
:1035D00094E00E94752F9B01AC01DC01CB010197A7
:1035E000A109B1090797A105B10508F08EC0A8EAA5
:1035F000B1E60E944F2E645E7C438E46944E05C019
:10360000611571058105910571F08B019C011457BD
:103610002B4832430130FAE51F07F2E62F07F2E0AC
:103620003F0708F05FC06093B1057093B2058093C7
:10363000B3059093B4053EC06F3F710581059105B8
:1036400011F008F04FC06093B50534C08B019C01A8
:1036500001501109210931090F3F110521053105DB
:1036600008F040C06093B60525C08B019C01045C46
:103670001940210931090D344DE1140721053105A7
:1036800028F47093B8056093B70514C061157105EF
:103690008105910521F48FEF8093B0050BC0613453
:1036A000710581059105F0F461506093B00502C089
:1036B000DD20C1F08091E00481111AC08091810564
:1036C00090918205A0918305B09184050196A11D7A
:1036D000B11D8093810590938205A0938305B093DB
:1036E000840506C06FE672E084EE95E00E94942A9D
:1036F0000E9403118FEF809347056AE084EE95E006
:103700000E94A62A0E940E1005C061E070E080E0D1
:1037100090E07BCF6C96E8E00C94ED2E6AE572E0C9
:1037200084EE95E00E94822A62E472E084EE95E0E5
:103730000E94822A84EE95E00E94A82B892B31F00A
:1037400084EE95E00E94D52B0E9407190E94DF1796
:10375000823029F0833051F46DE072E002C064E2FF
:1037600072E084EE95E00E94822A08958FEF8093A4
:1037700047051092E0040E940E10809147058E3F8D
:1037800069F084EE95E00E94A82B892BB1F384EEBA
:1037900095E00E94D52B0E940719EFCF08950F9353
:1037A0001F93109147051F3F09F0D2C0893409F4D7
:1037B00057C000F5883309F469C058F4803309F420
:1037C00077C008F061C08B3109F440C08132B1F19B
:1037D000B9C0813409F487C030F4893309F466C074
:1037E000803461F1AFC0823409F48EC0863409F4AC
:1037F00048C0A8C0823609F487C078F4883531F112
:1038000028F48235C1F18335E1F09CC08A3509F492
:1038100094C0813609F467C095C0823761F128F4FD
:10382000863679F18936E1F08DC0883779F08A37AC
:1038300009F483C0833709F085C003C060E172E0FA
:1038400015C00E943E0D6DE872E004C00E94470D55
:1038500067EA72E084EE95E00E94942A8EEF70C0D1
:103860000E947A060E94BF0666EC72E084EE95E044
:103870000E94942A67C081E00E94DF066FED72E02B
:10388000F5CF0E94B8105EC080535AC06AEF71E055
:1038900084EE95E00E94822A9091A00588E0890F2D
:1038A0008871977E892B8093A0051AC089E048C053
:1038B00067EE71E084EE95E00E94822A8091C10556
:1038C0009091C205A091C305B091C40520E1822763
:1038D0008093C1059093C205A093C305B093C4051E
:1038E000109347052FC061ED71E084EE95E00E94D2
:1038F000822A8091C1059091C205A091C305B09123
:10390000C40540E4842710C060EC71E084EE95E0CB
:103910000E94822A8091C1059091C205A091C305A1
:10392000B091C40520E282278093C1059093C2051F
:10393000A093C305B093C40502C00E948E1B8FEFF5
:1039400080934705809147058E3F09F0D4C0DDC0C4
:103950000E940D11882309F4D8C08091E1048111DF
:1039600004C08FEF80934705C6C040E050E060E0A0
:1039700070E082EE94E00E94752F009147051127B8
:1039800007FD1095212F312FF8013197E930F1050E
:1039900008F0B4C0E753FF4F0C94FE2E8B019C013E
:1039A000015014472B4832430F3F194522463240FD
:1039B00008F0A4C060937D0570937E0580937F0519
:1039C0009093800577C06093810570938205809302
:1039D00083059093840581E08093E0046BC0683098
:1039E00071058105910508F089C06093850562C065
:1039F0008B019C0101501109210931090A3011057F
:103A00002105310508F07AC06093860553C060EB4C
:103A100071E082EE94E00E94AF3010E0009799F0E0
:103A20000E948930009779F0183130F4E12FF0E0EE
:103A3000E858FA4F87871F5F60EB71E080E090E005
:103A40000E94AF30EBCF1831A8F5E12FF0E0E85835
:103A5000FA4F17861F5FF7CF653071058105910515
:103A600008F04CC060939F0525C08B019C0101505C
:103A70001109210931090630110521053105F0F53B
:103A80002091A005287F262B2093A00513C08B0131
:103A90009C0101501109210931090115124C2140E5
:103AA000310560F56093790570937A0580937B0505
:103AB00090937C058091E004811113C08091810571
:103AC00090918205A0918305B09184050196A11D76
:103AD000B11D8093810590938205A0938305B093D7
:103AE00084050E9403118FEF809347056AE084EEFE
:103AF00095E00E94A62A0E94821807C06FE672E035
:103B000084EE95E00E94942AECCF1F910F910895C6
:103B10008FEF809347051092E0040E9482188091F5
:103B200047058E3F69F084EE95E00E94A82B892B13
:103B3000B1F384EE95E00E94D52B0E94CF1BEFCF0E
:103B40006AE070E080E090E00E94E82884EE95E072
:103B50000E94A82B892B29F084EE95E00E94D52B9A
:103B6000F5CF0895CF93C82F682F84EE95E00E947B
:103B7000022C90916C059C2790936C05CF91089531
:103B8000A1E0B0E0E6ECFDE10C94D72E99830E9411
:103B9000B21D9981892F0E94B21D2196E2E00C94FA
:103BA000F32E1F93CF93DF93182FEB0110926C0528
:103BB00065EB70E084EE95E00E94590662E670E0E5
:103BC00084EE95E00E945906812F0E94B21DCE011D
:103BD0000E94C01DDF91CF911F91089560916C05E7
:103BE00084EE95E00E94022C0895A1E2B0E0EBEF94
:103BF000FDE10C94D32E7B018A018C3009F453C172
:103C000008F040C0863009F4BCC018F5833009F4D0
:103C100091C070F4813009F472C0823009F04AC258
:103C20006BE170E082E00E94D11D01EA15E078C0EE
:103C3000843009F487C0853009F03CC260914B059F
:103C400070E0660F771F85E00E94D11D0CE415E03F
:103C500086C0893009F4A7C070F4873009F49BC08E
:103C6000883009F027C261E070E088E00E94D11D31
:103C70008091D60525C28A3009F4CAC08B3009F478
:103C8000F2C018C28A3609F475C1D8F4873609F42F
:103C90003AC138F4853609F40EC1863609F41FC1DD
:103CA00009C2883609F437C1893609F003C261E0D8
:103CB00070E089E60E94D11D0E947A060E94BF062C
:103CC000F7C18D3609F4D4C138F48B3609F491C1AB
:103CD0008C3609F49AC1EEC18E3609F4DEC1873CF8
:103CE00009F0E8C161E070E087EC0E94D11D81E03D
:103CF0000E94B21D0E94EE1D10926D05E5C169E2A1
:103D000070E081E00E94D11D08E715E0F801819183
:103D10008F010E94B21DF5E0013A1F07B9F7D2C129
:103D2000F80181918F010E94B21DF5E00C3B1F0745
:103D3000B9F7C8C161E070E083E00E94D11D0E9424
:103D4000DF17BEC161E070E084E00E94D11D81E018
:103D50000E94B21D0E94EE1D0E941316B5C18091F3
:103D60004B0590E0880F991F98012C543540281777
:103D7000390708F0A7C1F80181918F010E94B21D97
:103D8000EECF62E070E086E00E94D11D88E893E00B
:103D90000E94C01D97C161E070E087E00E94D11DC4
:103DA00080914A058DC186E6898361E0CE01019646
:103DB0000E94DA0B0E94580B83E08093750568EC33
:103DC00070E080E090E00E94E828809175058430E2
:103DD000D9F48FE70E9476090E9489098983863485
:103DE00069F460E270E089E00E94D11D10E20E9457
:103DF00089090E94B21D1150D1F764C161E070E0E1
:103E000089E00E94D11D54C161E070E089E055C194
:103E100069E170E08AE00E94D11D81E08093BC05D9
:103E2000209174058091C1059091C205A091C305B0
:103E3000B091C405222311F0806801C08F77809370
:103E4000C1059093C205A093C305B093C4050CEBC4
:103E500015E0F80181918F010E94B21DF5E0053D4A
:103E60001F07B9F72FC161E270E08BE00E94D11DFE
:103E70008091A8048F3F39F08091A80491E0980FB9
:103E80009093A80402C08091A8040E94B21D10E083
:103E9000812F0E94DA150E9409090E94C01D1F5F30
:103EA0001031B1F70FC161E070E08CE00E94D11DCC
:103EB0008091D50505C161E070E085E60E94D11DC5
:103EC00089E2E816F10409F0FAC0D801E8E7F5E064
:103ED0008D91819385E0E13AF807D1F7E9C061E07F
:103EE00070E086E60E94D11DEBE1EE16F10409F0C8
:103EF000E6C0D801E1EAF5E08D91819385E0EC3BE5
:103F0000F807D1F7D5C061E070E087E60E94D11DC7
:103F10000E943E0DCDC061E070E088E60E94D11D98
:103F200085E789838BE1E1EAF5E0DE0112960190F5
:103F30000D928A95E1F76CE1CE0101960E94DA0BB1
:103F40000E94580B83E08093750560E273E080E087
:103F500090E00E94E82880917505843009F0AFC098
:103F60008FE70E9476090E9489098983853509F0C7
:103F7000A6C09EC061E070E08AE60E94D11D89E67D
:103F8000898361E0CE0101960E94DA0B0E94580BF2
:103F900083E08093750560E273E080E090E00E942A
:103FA000E82880917505843009F089C08FE70E9468
:103FB00076090E94890989838E010E5F1F4F7E0159
:103FC000EDE1EE0EF11C0E948909F80181938F0149
:103FD000EE15FF05C1F78BE1FE013296A1EAB5E0CF
:103FE00001900D928A95E1F78981893409F067C0C3
:103FF0005FC061E070E08BE60E94D11DF801808116
:104000008093D6050E94470D53C061E070E08CE6B6
:104010000E94D11DF0E2EF16F10461F487E6898376
:1040200080E2F801DE01129601900D928A95E1F787
:1040300061E203C087E4898361E0CE0101960E94BA
:10404000DA0B0E94580B83E0809375056CE474E0F2
:1040500080E090E00E94E82880917505843079F531
:104060008FE70E9476090E948909873441F520C0B4
:1040700061E070E08DE60E94D11D89E1E816F1044F
:10408000F1F4D801ECEBF5E08D91819385E0E53D0D
:10409000F807D1F70E9491130BC061E070E08EE643
:1040A0000E94D11DF80180818093D5050E94280DC2
:1040B00081E006C061E070E08AEC0E94D11D80E0E2
:1040C0000E94B21D0E94EE1DA196E6E00C94EF2E18
:1040D000A0E0B0E0EEE6F0E20C94D12ECAECD3E022
:1040E00014E606E035E0F32E44E0E42E53E0D52E4E
:1040F00062E0C62E84EE95E00E94A82B892B09F47D
:104100009BC084EE95E00E94D52B282F8093350428
:104110004091340450E04730510560F7FA01EE5207
:10412000FF4F0C94FE2E853B29F781E080933404E9
:10413000E1CF823609F07DC0C0923404DBCF80939A
:10414000330480933204D0923404D4CF9C013327BB
:104150003093310420933004909132049827909347
:104160003204E0923404C6CF382F22274091300425
:1041700050913104242B352B30933104209330049B
:1041800090913204982790933204F09234042536AB
:10419000310508F4AFCF61E070E08CEC0E94D11DD6
:1041A00081E00E94B21D0E94EE1D43C020912E04AA
:1041B00030912F04F901E653FC4F80839091320433
:1041C000982790933204C901019690932F0480930D
:1041D0002E0420913004309131048217930708F4A3
:1041E00089CF0093340486CF8091320482130BC0B0
:1041F00060912E0470912F044AEC53E080913304B7
:104200000E94F51D0DC062E070E08BEC0E94D11D94
:10421000809133040E94B21D80916C050E94B21DF2
:10422000FE01812F11928A95E9F710922F041092C6
:104230002E04109234045ECFCDB7DEB7E8E00C94C4
:10424000ED2E81E080936D0580916D05882349F006
:1042500084EE95E00E94A82B892BB1F30E94682080
:10426000F3CF0895AAE2B0E0E8E3F1E20C94CF2E98
:104270000E94B9286B017C0181E00E947D0A84EED6
:1042800095E00E94A82B892B29F084EE95E00E94EE
:10429000D52BF5CF2C9811E072E6B72EE9E2AE2EC1
:1042A00003E00E94B9286C197D098E099F09693CB9
:1042B000710581059105D0F11123C1F10E94B92842
:1042C0006B017C012B9A80ED97E00E94A807B982D0
:1042D000E8E7F5E0DE0112968A2D01900D928A95AD
:1042E000E1F76AE2CE0101960E94DA0B2B9880E09A
:1042F00090E00E94A807009375050E94580B62E3A6
:1043000070E080E090E00E94E8288091750584309C
:1043100061F4009375058FE70E9476090E94890970
:1043200011E0823419F410E001C011E08AE00E942B
:10433000DE29892B81F411E00EC02C9A2B9A84EE91
:1043400095E00E94D52B8D309105A9F05CF40A9779
:1043500091F02C982B9884EE95E00E94A82B892B45
:1043600061F79FCF8332910579F08234910589F707
:104370000E942121EECF62EB71E084EE95E00E9475
:10438000822A0E94881DE5CF0E941316E2CF8F92E9
:104390009F92AF92BF92CF92DF92EF92FF921F93C4
:1043A000CF93DF938AE00E94DE29892B09F089C030
:1043B00068EC70E080E090E00E94E82880E090E007
:1043C0000E94A8070E94B9284B015C016B017C0187
:1043D00080ECC80E82E1D81EE11CF11C0E94B928B5
:1043E0006C157D058E059F0530F48AE00E94DE295C
:1043F000892BA1F364C08AE00E94DE29892B09F091
:104400005EC080ED97E00E94A8070E94B9286B016A
:104410007C01D0E0C1E088E4880E86E2981EA11CF1
:10442000B11C11E08AE00E94DE29892B21F58C1451
:104430009D04AE04BF0430F480ED97E00E94A8070D
:10444000D1E0F0CF0E94B9286C197D098E099F092F
:10445000693C71058105910528F30E94B9286B011B
:104460007C01C12719F080ED97E002C080E090E068
:104470000E94A807D7CF80E090E00E94A807DD2324
:10448000B9F08091D50590E0019665E070E00E945A
:10449000722E8093D5050E94280D0E94A8130E94B9
:1044A000470D64EF71E080E090E00E94E82809C0C9
:1044B00080E00E94DF060E94BF110E943E0D0E9414
:1044C0003221DF91CF911F91FF90EF90DF90CF903D
:1044D000BF90AF909F908F900895CF92DF92EF9210
:1044E000FF9280E00E94DA070E94B10761E08CE051
:1044F0000E94722961E08BE00E94722960E08AE0EC
:104500000E94722960E083E10E94722961E083E1E8
:104510000E94AB2961E082E10E94722960E082E1A1
:104520000E94AB290E949F0740E052EC61E070E0DE
:1045300084EE95E00E94F02C0E94A8130E94470D83
:104540000E9491138FEF8093A8040E94C60778946D
:104550000E94B9286B017C018091A8048F3F59F417
:104560000E94B9286C197D098E099F09603D77402A
:104570008105910588F380ED97E00E94A80761E02E
:104580008AE00E94AB292C9A84EE95E00E94A82B29
:10459000892B29F084EE95E00E94D52BF5CF6CEFA6
:1045A00072E084EE95E00E94632A88E893E00E941E
:1045B0002F0C63E173E084EE95E00E94632A4AE0E9
:1045C00050E060E070E084EE95E00E94332B62E3FF
:1045D00070E080E090E00E94E82884EE95E00E9480
:1045E000A82B04970CF184EE95E00E94D52B823421
:1045F0009105D1F484EE95E00E94D52B8E3491057F
:1046000099F484EE95E00E94D52B8434910561F4F1
:1046100084EE95E00E94D52B819731F480E090E004
:104620000E94A8070E9432214091790550917A0595
:1046300060917B0570917C05DB01CA010197A1099E
:10464000B1090497A105B10590F44093A704433044
:1046500051F42EE240EA56E861E070E084EE95E025
:104660000E94712D08C040E052EC61E070E084EEE1
:1046700095E00E94F02C0E94C7212C9880E090E0E9
:104680000E94A8070E9491131092C7048091C1054F
:1046900083FF11C080918D05882351F0809194058E
:1046A000882331F080919B05882311F087E001C0B9
:1046B00085E08093C70480E00E947D0A8091C80451
:1046C0000E94B1090E94580B10923F0410923E04C0
:1046D00010923D04F12C8091D6058F15B0F062E365
:1046E00070E080E090E00E94E82880ED97E00E9472
:1046F000A80762E370E080E090E00E94E82880E094
:1047000090E00E94A807F394E6CF8091A00584FF73
:1047100008C0982F987181E0983109F080E00E94DC
:104720007B118FE00E94DA07FF90EF90DF90CF902F
:104730000895EF92FF920F931F93CF93DF938C0115
:104740006EE770E084EE95E00E945906E801F12CD6
:10475000F0E2EF2E8E0188818D57823048F46DE7AC
:1047600070E084EE95E00E94590688818E2588834A
:104770002196F801608184EE95E00E94022CF3946A
:10478000F9E0FF12E7CF6EE770E084EE95E00E945B
:104790005906CDB7DEB7E6E00C94EF2EA9E0B0E005
:1047A000E4EDF3E20C94D72E9091C90491110EC060
:1047B0009EEF99838A836B8350E0559547954C8390
:1047C0002D83198618861F821E822EC04091CE042A
:1047D000842F90E0B4E095958795BA95E1F7242F62
:1047E0002F7030E08217930719F18DEF89831B82B8
:1047F000FE01349650E0842F90E0A4E095958795D3
:10480000AA95E1F7242F2F7030E08217930749F023
:10481000DC01A153BB4F8C918193405F5F5F5630A9
:1048200051F74093CE045A83CE0101960E949923FA
:104830008091C90490E0019666E070E00E94722EBB
:104840008093C9042996E2E00C94F32EA0E0B0E036
:10485000ECE2F4E20C94D02E6C016EE770E084EE92
:1048600095E00E9459068601E12CF12CC0E0D0E0D1
:1048700030E2B32EF801608183E8860F823078F44D
:104880006DE770E084EE95E00E945906F8016081C2
:104890006B2570E084EE95E00E94590604C084EE1A
:1048A00095E00E94022CE114F10459F0F801808196
:1048B0009E01280F311DC901C92FDD27C80FD91F3F
:1048C000DD273FEFE31AF30A89E0E816F10459F017
:1048D00028E0E216F10421F48C2F8095F601808700
:1048E0000F5F1F4FC7CFCDB7DEB7E9E00C94EC2EBA
:1048F000A9E0B0E0EEE7F4E20C94D72EE82F362FD3
:104900008091C90490E0019664E270E00E94722EEA
:104910008093C90458E9598350E15A83813089F062
:1049200048F08230B9F08330D9F48B8381EF8C83E7
:104930003D8319C085E08B8381EF8C832F5F2D83AE
:1049400012C08B8381EF8C8384E6489FA0011124E1
:104950005D8309C084E08B8381EF8C83ED8303C08A
:104960000E94B81104C0CE0101960E942624299607
:10497000E2E00C94F32EA2E0B0E0E1ECF4E20C945F
:10498000CC2E182F762E2A8349830E94C5286B01CE
:104990007C018091DF048090CA049090CB04A090A9
:1049A000CC04B090CD042A8149818823C1F0D7017D
:1049B000C60188199909AA09BB094C015D0191EE4C
:1049C00089169EE29906A104B10420F1241708F487
:1049D000422F202F672D812F0E94782413C0D701EA
:1049E000C60188199909AA09BB094C015D0191E327
:1049F000891695E79906A104B10460F0672D812F0F
:104A00000E94CE23C092CA04D092CB04E092CC0480
:104A1000F092CD042296EDE00C94E82EA2E2B0E0F4
:104A2000E4E1F5E20C94CD2E8CE00E94980981110E
:104A30000DC06BE173E084EE95E00E94942A2C9AFD
:104A400080E00E947D0A0E94580B2C9884EE95E02D
:104A50000E94A82B892B01F184EE95E00E94D52BB2
:104A60009091A704992319F00E94BB13EFCF4091B6
:104A70003E0450E09A012F5F3F4F2F713327609122
:104A80003F0470E02617370709F3FA01E75BFB4F95
:104A9000808320933E04DACF80917505843009F03D
:104AA00086C00E94C528611571058105910549F0F0
:104AB0006093B9047093BA048093BB049093BC04D0
:104AC0000CC081E090E0A0E0B0E08093B904909346
:104AD000BA04A093BB04B093BC048091AB04909142
:104AE000AC0481609093AC048093AB0483E080932A
:104AF00075058FE70E94760909E614E00E9489098E
:104B0000F80181938F01F4E002371F07B9F7209174
:104B1000720480916904982F922796FF3BC090E41D
:104B2000922790937204982F98739833F1F410E0C1
:104B3000212F30E080916904877090E082179307FD
:104B40004CF11F5F2091A005812F90E0FC01E759F7
:104B5000FB4F24FF04C080810E949A11E9CF60813D
:104B600084EE95E00E94022CE3CF8F7399F480913C
:104B70006A048093B40480916B048093B2048091A2
:104B80006C048093B10480916F0490E09093AA0428
:104B90008093A90480913D04813019F482E08093D0
:104BA0003D0480913D04833011F410923D040E9435
:104BB000C5286B017C018091AD049091AE04A09159
:104BC000AF04B091B0040097A105B105C9F0A701E9
:104BD0009601281B390B4A0B5B0BDA01C901883B94
:104BE0009B40A105B10560F00E94C7098093B30402
:104BF0001092AD041092AE041092AF041092B00463
:104C00008091BD049091BE04A091BF04B091C004F6
:104C100046015701881A990AAA0ABB0A88E795E053
:104C20000E94F40786169706A806B90608F4A8C0DD
:104C3000C092BD04D092BE04E092BF04F092C004C2
:104C40000E9457068091A8048830A0F08091C10589
:104C50009091C205A091C305B091C4055CE1B695E1
:104C6000A795979587955A95D1F7892B8A2B8B2BEA
:104C700009F0AAC18091A8048F5F8093A804809155
:104C8000B9049091BA04A091BB04B091BC04009700
:104C9000A105B105F1F0C81AD90AEA0AFB0A88E7AA
:104CA00095E00E94F4076C157D058E059F0508F0C0
:104CB00012C18091C10584FD04C080ED97E00E947F
:104CC000A8071092B9041092BA041092BB04109273
:104CD000BC0490917204907C9093720450913E04B5
:104CE00080913F0420913D04581709F411C12230EE
:104CF00009F00EC1905890937204E091A005E770FE
:104D0000F0E0E758FC4F6081693008F0E9C061507D
:104D100040E04613E7C080933F0487E3840F9091FF
:104D20007204892B809372044093400483E0809343
:104D30003D042B9A809185059091C704911135C14E
:104D40000E94780A8091C8040E94B109E091A005F0
:104D5000E770F0E0E758FC4F608182E794E00E9442
:104D6000930BE091C804EF5FE093C804E83109F4C5
:104D700028C1F0E0E858FA4F8785882309F421C15B
:104D80000E94020C813069F58091A005887149F17B
:104D90008091AB049091AC04880F991F9093AC0460
:104DA0008093AB0483E0809375050E94580B0E94AA
:104DB000C5286093AD047093AE048093AF049093C4
:104DC000B004672B682B692B61F481E090E0A0E0D0
:104DD000B0E08093AD049093AE04A093AF04B09381
:104DE000B0048091A00584FF2BC08091B9049091FC
:104DF000BA04A091BB04B091BC04892B8A2B8B2BE5
:104E0000F9F08091AB049091AC048E7F0E942A0946
:104E1000182F6091A9048091B4040E94B113482F07
:104E2000612F8091B30449A30E94B1130091D6056C
:104E3000282F49A16091B1048091B2040E94BB2443
:104E40002B988091C5048130C1F018F08230B1F107
:104E5000C8C08AE00E94DE29892B09F0C2C081E027
:104E60008093C5040E94B9286093C1047093C20462
:104E70008093C3049093C404B4C08AE00E94DE29E6
:104E8000892B31F50E94B928C090C104D090C2048A
:104E9000E090C304F090C4046C197D098E099F0949
:104EA000693E73408105910508F49BC082E08093C0
:104EB000C50480ED97E00E94A80793C08AE00E9495
:104EC000DE29892B09F48DC080E090E00E94A807BC
:104ED0001092C50486C080E090E00E94A807F9CE39
:104EE00068E016CF851709F416CF4F5F242F30E006
:104EF00090E0F901EE58FB4FDC01A75BBB4F7C91C2
:104F00007083F901E05CFB4F708301968F7101CFD4
:104F10002430B1F42091400481E494E0A3E7B4E0AC
:104F2000FC013E2F381B321718F431913D93F9CF15
:104F300087E3820F90917204892B80937204F6CEDE
:104F40008091C504823051F49160909372042C9A40
:104F50008E010F5F1F4FF12CB80110C02C9880916B
:104F60003D04811103C081E080933D0480913D04A4
:104F7000833071F784E080933D04EACF8F2D69A3DD
:104F80007AA30E94DA15F801819391938F01F3942B
:104F900069A17AA1F0E1FF12F1CF8091A00543E76A
:104FA00054E087700E947908C4CE882309F4C8CEE3
:104FB0002091C60431E0320F3093C6042913C0CECD
:104FC0000CC01092C804DCCE8091A804883009F48B
:104FD0002C9A89E08093A804D3CE1092C604815005
:104FE000AFCEA296ECE00C94E92E8230E8F4E82FE4
:104FF000F0E0EE0FFF1FE952FA4F718360838130BA
:1050000041F0809169008C7F842B80936900E89A3D
:10501000089580916900440F551F440F551F837FE9
:10502000842B80936900E99A08951F920F920FB61E
:105030000F9211242F933F934F935F936F937F931E
:105040008F939F93AF93BF93EF93FF938091D70577
:105050009091D805892B29F0E091D705F091D805DA
:105060000995FF91EF91BF91AF919F918F917F91A2
:105070006F915F914F913F912F910F900FBE0F90C5
:105080001F9018951F920F920FB60F9211242F9315
:105090003F934F935F936F937F938F939F93AF93C0
:1050A000BF93EF93FF938091D9059091DA05892BF7
:1050B00029F0E091D905F091DA050995FF91EF917A
:1050C000BF91AF919F918F917F916F915F914F9120
:1050D0003F912F910F900FBE0F901F9018951F9228
:1050E0000F920FB60F9211242F933F938F939F939C
:1050F000AF93BF938091DC059091DD05A091DE0513
:10510000B091DF053091DB0523E0230F2D3720F42C
:105110000196A11DB11D05C026E8230F0296A11D11
:10512000B11D2093DB058093DC059093DD05A093F2
:10513000DE05B093DF058091E0059091E105A09137
:10514000E205B091E3050196A11DB11D8093E00534
:105150009093E105A093E205B093E305BF91AF9171
:105160009F918F913F912F910F900FBE0F901F90A5
:1051700018952FB7F8946091DC057091DD0580914A
:10518000DE059091DF052FBF08953FB7F894809119
:10519000E0059091E105A091E205B091E30526B507
:1051A000A89B05C02F3F19F00196A11DB11D3FBF5F
:1051B0006627782F892F9A2F620F711D811D911DEF
:1051C00042E0660F771F881F991F4A95D1F708950F
:1051D000CF92DF92EF92FF92CF93DF936B017C012E
:1051E0000E94C528EB01C114D104E104F10479F057
:1051F0000E94C5286C1B7D0B683E7340A0F381E0C4
:10520000C81AD108E108F108C851DC4FECCFDF9192
:10521000CF91FF90EF90DF90CF900895789484B570
:10522000826084BD84B5816084BD85B5826085BDA2
:1052300085B5816085BDEEE6F0E080818160808388
:10524000E1E8F0E01082808182608083808181606B
:105250008083E0E8F0E0808181608083E1EBF0E032
:10526000808184608083E0EBF0E0808181608083D6
:10527000EAE7F0E0808184608083808182608083BF
:105280008081816080838081806880831092C100EA
:105290000895833081F028F4813099F08230A1F0B4
:1052A00008958630A9F08730B9F08430D1F4809128
:1052B00080008F7D03C0809180008F778093800075
:1052C000089584B58F7702C084B58F7D84BD08951D
:1052D0008091B0008F7703C08091B0008F7D809364
:1052E000B0000895CF93DF9390E0FC01ED50F44FB0
:1052F0002491FC01E95FF34F8491882349F190E008
:10530000880F991FFC01E15DF34FA591B4918B5D6E
:10531000934FFC01C591D4919FB7611108C0F894D7
:105320008C91209582238C93888182230AC06230DD
:1053300051F4F8948C91322F309583238C9388818B
:10534000822B888304C0F8948C91822B8C939FBF0E
:10535000DF91CF910895A1E0B0E0E1EBF9E20C9488
:10536000D52E282F30E0F901E152F44F8491F90154
:10537000ED50F44F1491F901E95FF34F04910023CC
:10538000C9F0882321F069830E9449296981E02FAF
:10539000F0E0EE0FFF1FEB5DF34FA591B4919FB7C7
:1053A000F8948C91611103C01095812301C0812B69
:1053B0008C939FBF2196E4E00C94F12ECF93DF9362
:1053C000282F30E0F901E152F44F8491F901ED50BA
:1053D000F44FD491F901E95FF34FC491CC2391F0DC
:1053E00081110E944929EC2FF0E0EE0FFF1FE55ECE
:1053F000F34FA591B4912C912D2381E090E021F4FD
:1054000080E002C080E090E0DF91CF910895A0E0BD
:10541000B0E0EDE0FAE20C94D12E6C017A01EB01E0
:10542000E60EF71E00E010E0CE15DF0561F0699191
:10543000D601ED91FC910190F081E02DC601099516
:10544000080F191FF1CFC801CDB7DEB7E8E00C9403
:10545000ED2E6115710589F0DB010D900020E9F753
:10546000AD0141505109461B570BDC01ED91FC91F8
:105470000280F381E02D0995089580E090E0089581
:10548000EF92FF920F931F93CF93DF938C01FB0159
:10549000C0E0D0E064917F018FEFE81AF80A66233C
:1054A00061F0D801ED91FC910190F081E02DC801EF
:1054B0000995C80FD91FF701EDCFCE01CDB7DEB7E3
:1054C000E6E00C94EF2E0E94292A0895DC01ED916C
:1054D000FC910190F081E02D099508950F931F93A1
:1054E000CF93DF93EC016DE00E94662A8C016AE0A5
:1054F000CE010E94662A800F911FDF91CF911F91EC
:105500000F9108950F931F93CF93DF93EC010E94A7
:10551000402A8C01CE010E946E2A800F911FDF91DC
:10552000CF911F910F9108950F931F93CF93DF9306
:10553000EC010E94292A8C01CE010E946E2A800F64
:10554000911FDF91CF911F910F9108950F931F939A
:10555000CF93DF93EC010E94662A8C01CE010E945A
:105560006E2A800F911FDF91CF911F910F910895A7
:10557000A1E2B0E0EEEBFAE20C94CD2E7C01C42E59
:10558000E52FCB01D22E19A221E02D1510F02AE033
:10559000D22E8E010F5D1F4F8D2C912CA12CB12C82
:1055A0006C2D7E2FA50194010E94862E8C2DD29EFB
:1055B00080191124015011098A3010F4805D01C056
:1055C000895CF8018083211531054105510521F0E1
:1055D000C22EE32FCA01E4CFB801C7010E94292AD5
:1055E000A196ECE00C94E92EA0E0B0E0EAEFFAE23C
:1055F0000C94D12EEC016A017B012115310541F497
:10560000E881F9810190F081E02D642F09951DC09A
:105610002A303105A9F477FF12C06DE20E94662A94
:105620008C0144275527BA014C195D096E097F0981
:105630002AE0CE010E94B82A800F911F06C02AE0FE
:10564000B701A601CE010E94B82ACDB7DEB7E8E0C7
:105650000C94ED2E9A01AB01662757FD6095762FCD
:105660000E94F42A08950F931F93CF93DF93EC01C8
:105670009A01AB01662757FD6095762F0E94F42AA8
:105680008C01CE010E946E2A800F911FDF91CF9175
:105690001F910F9108952115310549F4DC01ED9119
:1056A000FC910190F081E02D642F099508950E94EE
:1056B000B82A08959A01462F50E060E070E00E94F9
:1056C0004B2B08959A01AB0160E070E00E944B2BD8
:1056D00008950F931F93CF93DF93EC010E944B2B00
:1056E0008C01CE010E946E2A800F911FDF91CF9115
:1056F0001F910F9108950F931F93CF93DF93EC01A8
:105700009A01AB0160E070E00E944B2B8C01CE014E
:105710000E946E2A800F911FDF91CF911F910F91F0
:1057200008950F931F93CF93DF93EC019A01462FB7
:1057300050E060E070E00E944B2B8C01CE010E9493
:105740006E2A800F911FDF91CF911F910F910895C5
:10575000FC0124853585F901E05CFF4F8081918152
:10576000F901EE5BFF4F20813181821B930B8F7318
:1057700099270895FC0184859585FC01E05CFF4F25
:1057800040815181FC01EE5BFF4F20813181421746
:10579000530741F00190F081E02DE80FF91F80815F
:1057A00090E008958FEF9FEF0895FC018485958523
:1057B000FC01E05CFF4F40815181FC01EE5BFF4F3B
:1057C000208131814217530779F0A081B181A80F60
:1057D000B91F8C91208131812F5F3F4F2F73332769
:1057E0003183208390E008958FEF9FEF0895FC01AF
:1057F00081A1882329F0A489B5898C9186FFFBCFEC
:1058000011A20895CF93DF93FC0126853785D90136
:10581000A05CBF4F8D919C91119701968F73992732
:10582000E901CE5BDF4F4881598184179507D9F391
:105830000D90BC91A02DA20FB31F6C93A685B785C8
:10584000A05CBF4F11969C938E93A689B7892C912B
:1058500081E090E0078C02C0880F991F0A94E2F75C
:10586000282B2C9381E081A30488F589E02D808189
:105870008064808381E090E0DF91CF910895089566
:105880001F920F920FB60F9211242F933F934F93B5
:105890008F939F93EF93FF938091C00082FD1CC074
:1058A0004091C60080918A0690918B0601968F7375
:1058B000992720918C0630918D068217930771F0FD
:1058C000E0918A06F0918B06E65BF94F4083909356
:1058D0008B0680938A0602C08091C600FF91EF91EB
:1058E0009F918F914F913F912F910F900FBE0F90ED
:1058F0001F90189584EE95E00E94A82B892B11F03B
:105900000E943F2C08951F920F920FB60F92112400
:105910002F933F938F939F93EF93FF93209146068E
:10592000309147068091480690914906281739071B
:1059300031F48091C1008F7D8093C10014C0E0914B
:105940004806F0914906EA5FF94F208180914806A8
:105950009091490601968F739927909349068093F9
:1059600048062093C600FF91EF919F918F913F9140
:105970002F910F900FBE0F901F901895A0E0B0E0F0
:10598000E4ECFCE20C94CD2EFC011382128288EE32
:1059900093E0A0E0B0E084839583A683B7838BEB8C
:1059A00093E0918380837587648757874687318B1F
:1059B000208B138B028BF58AE48AD78AC68AB18E34
:1059C000A08E938E828E8F85848F8889858F89891A
:1059D000868F8A89878F8B8980A3ECE00C94E92ECF
:1059E000CF92DF92EF92FF92CF93DF93EC016A01A7
:1059F0007B01411581EE580761057105F9F0EC89CD
:105A0000FD8981E090E008A002C0880F991F0A94E8
:105A1000E2F7808360E079E08DE390E0A7019601F2
:105A20000E94862E2150310941095109569547950A
:105A300037952795211580E1380798F0EC89FD8985
:105A4000108260E874E88EE190E0A70196010E9460
:105A5000862E2150310941095109569547953795B0
:105A60002795E889F9893083EA89FB89208319A27F
:105A7000EE89FF89408181E090E09C010C8C02C09E
:105A8000220F331F0A94E2F7422B4083EE89FF89ED
:105A900040819C010D8C02C0220F331F0A94E2F753
:105AA000422B4083EE89FF8940819C010E8C02C00D
:105AB000220F331F0A94E2F7422B4083EE89FF89BD
:105AC00020810F8C02C0880F991F0A94E2F78095FD
:105AD00082238083DF91CF91FF90EF90DF90CF9072
:105AE0000895BF92CF92DF92EF92FF92CF93DF9310
:105AF000EC016A017B01B22E411581EE5807610568
:105B00007105F9F0EC89FD8981E090E008A002C000
:105B1000880F991F0A94E2F7808360E079E08DE3B3
:105B200090E0A70196010E94862E2150310941097B
:105B300051095695479537952795211580E13807E6
:105B400098F0EC89FD89108260E874E88EE190E0BD
:105B5000A70196010E94862E215031094109510961
:105B60005695479537952795E889F9893083EA89CD
:105B7000FB892083E88DF98DB082EE89FF89408111
:105B800081E090E09C010C8C02C0220F331F0A942C
:105B9000E2F7422B4083EE89FF8940819C010D8C06
:105BA00002C0220F331F0A94E2F7422B4083EE8992
:105BB000FF8940819C010E8C02C0220F331F0A9482
:105BC000E2F7422B4083EE89FF8920810F8C02C0CF
:105BD000880F991F0A94E2F7809582238083DF91D2
:105BE000CF91FF90EF90DF90CF90BF9008958F926C
:105BF0009F92AF92BF92CF92DF92EF92FF920F935C
:105C00001F9381E08F9385E08F9387E08F9383E0EC
:105C10008F9384E08F93E6EC8E2E912CF2ECAF2ED6
:105C2000B12CA1ECCA2ED12CB0ECEB2EF12C04EC53
:105C300010E025EC30E046E056E06AE476E084EEE1
:105C400095E00E94BE2C0F900F900F900F900F9038
:105C50001F910F91FF90EF90DF90CF90BF90AF908A
:105C60009F908F9008950E940E290E946D22CAE78E
:105C7000DCE20E940E252097E1F30E947A2CF9CFF6
:105C8000A29FB001B39FC001A39F700D811D11247D
:105C9000911DB29F700D811D1124911D08950E94C8
:105CA000402EA59F900DB49F900DA49F800D911D37
:105CB00011240895B7FF0C944F2E0E944F2E821B83
:105CC000930B0895DB018F939F930E944F2EBF91FA
:105CD000AF91A29F800D911DA39F900DB29F900D3B
:105CE0001124089597FB072E16F4009407D077FD32
:105CF00009D00E94042F07FC05D03EF490958195B1
:105D00009F4F0895709561957F4F0895A1E21A2ED7
:105D1000AA1BBB1BFD010DC0AA1FBB1FEE1FFF1F4F
:105D2000A217B307E407F50720F0A21BB30BE40B9F
:105D3000F50B661F771F881F991F1A9469F76095E6
:105D40007095809590959B01AC01BD01CF010895A0
:105D5000052E97FB1EF400940E94BF2E57FD07D01E
:105D60000E94862E07FC03D04EF40C94BF2E509553
:105D70004095309521953F4F4F4F5F4F0895909537
:105D80008095709561957F4F8F4F9F4F08952F920B
:105D90003F924F925F926F927F928F929F92AF92BB
:105DA000BF92CF92DF92EF92FF920F931F93CF9308
:105DB000DF93CDB7DEB7CA1BDB0B0FB6F894DEBF9F
:105DC0000FBECDBF09942A88398848885F846E84C5
:105DD0007D848C849B84AA84B984C884DF80EE800F
:105DE000FD800C811B81AA81B981CE0FD11D0FB618
:105DF000F894DEBF0FBECDBFED010895EE0FFF1F7B
:105E00000590F491E02D0994AA1BBB1B51E107C03A
:105E1000AA1FBB1FA617B70710F0A61BB70B881F3A
:105E2000991F5A95A9F780959095BC01CD010895C9
:105E30008F929F92AF92BF92CF92DF92EF92FF929A
:105E4000CF93DF93EC01688179818A819B81611511
:105E500071058105910521F464E279ED8BE597E008
:105E60002DE133EF41E050E00E94A82E49015A0194
:105E70009B01AC01A7EAB1E40E944F2E6B017C01AB
:105E8000ACEEB4EFA50194010E945D2EC60ED71EA4
:105E9000E81EF91EF7FE06C081E0C81AD108E10825
:105EA00080E8F80AC882D982EA82FB82C701B6017B
:105EB0009F77DF91CF91FF90EF90DF90CF90BF90D1
:105EC000AF909F908F9008950E94182F089586E0BC
:105ED00091E00E94182F08956093060170930701C6
:105EE000809308019093090108952F923F925F9249
:105EF0006F927F928F929F92AF92BF92CF92DF92DA
:105F0000EF92FF920F931F93CF93DF938B01EA01E0
:105F10006115710521F0DB018C9311969C932097FC
:105F200039F09E01225031092332310508F0D8C0E2
:105F30007C016701BFEFCB1ADB0A5601F7016080D5
:105F4000862D90E00E94A730892B11F07601F1CFC9
:105F5000FDE26F120AC0570182E0A80EB11CD70102
:105F600011966C90772473940BC0BBE26B1207C040
:105F70005701E2E0AE0EB11CD70111966C90712C66
:105F8000CE018F7E892B89F4B0E36B1237C0F50107
:105F900080818F7D8835D1F46180F2E0AF0EB11C35
:105FA000872D8260782EC0E1D0E0CA30D10551F152
:105FB000C031D10521F0C830D10599F409C0CC24F5
:105FC000CA94DC2CEC2CAFE0FA2E22C0209769F7A3
:105FD000C8E0D0E0CC24CA94DC2CEC2CFFE1FF2EEE
:105FE00017C06FEF7FEFCB019E01442737FD40952F
:105FF000542F0E94862E69017A010AC02097A9F6C3
:10600000CAE0D0E0E9E9CE2EDC2CEC2CE9E1FE2E52
:10601000F50160E020E030E0A9014E01AA2497FCE0
:10602000A094BA2C1F0170ED572E560CA9E0A515AF
:1060300070F48FEB860D8A3118F499EC592E06C056
:106040008FE9860D8A3148F589EA582E560C852D40
:1060500090E08C179D070CF56F3FD9F0C216D30660
:10606000E406F50698F0C501B4010E94622E9B017A
:10607000AC01852D90E0A0E0B0E0280F391F4A1F49
:106080005B1F281739074A075B0710F46FEF01C041
:1060900061E03196D1016C90C5CF0115110551F029
:1060A000662311F0319703C071FE04C03297D80106
:1060B000ED93FC9370FE07C0509540953095219567
:1060C0003F4F4F4F5F4F67FF10C082E290E09093C9
:1060D0008F0680938E066FEF7FEF8FEF9FEF07C0E5
:1060E00060E070E080E090E002C0B901CA01DF9199
:1060F000CF911F910F91FF90EF90DF90CF90BF90C5
:10610000AF909F908F907F906F905F903F902F9077
:106110000895FC0188279927E89421912032E9F31A
:10612000293010F02E30C8F32B3241F02D3239F4E3
:10613000689404C00E94DB30820F911D219120538E
:106140002A30C0F31EF4909581959F4F08959111C8
:1061500050C0803219F089508550D0F7089548EC2E
:1061600053E00E94B4300895FA01A191B0810097E4
:1061700019F41097E1F0CD01DC01CD010D90002064
:1061800011F4C00113C0FB012191222319F0201545
:10619000D9F7F3CFFB012191201519F41E92119626
:1061A00006C02223C1F70D900020A1F7D001FA010B
:1061B000A193B08308957AE0979F902D879F802DBB
:1061C000910D11240895F999FECF92BD81BDF89AE1
:1061D000992780B50895262FF999FECF1FBA92BD51
:1061E00081BD20BD0FB6F894FA9AF99A0FBE0196B8
:0C61F0000895992788270895F894FFCFA0
:1061FC0000009006200001000000FF0002000200D9
:10620C000200020002000200020002000200020072
:10621C0002000200020002000200028025000005BC
:10622C00400AA1204EA50020244EA52C2330C012DC
:10623C0000001A400AA1204EA5001B1E27522C2339
:10624C00308025000005400AA1204EA50020244ED8
:10625C00A52C2330004B000006400AD0009D4900BD
:10626C007B289D492C233000E1000005400A4501A4
:10627C00D7DC03B81E0EBF00232E48E801008A406D
:10628C000A6001555502AD1E20000023C854582049
:10629C0074696D656F75742100596573004E6F00DC
:1062AC002C00386368004E2F41002C205B005D20D1
:1062BC0028002900486F70206368616E6E656C2041
:1062CC000020402000456E746572696E6720616421
:1062DC00617074697665206368616E6E656C20739D
:1062EC00656C656374696F6E2C207069636B696E85
:1062FC00673A007363616E6E6572206D6F64650042
:10630C004E4F5420454E41424C45440053656E64FB
:10631C00696E672073657474696E677320746F207F
:10632C0052580A00526573657474696E6720736500
:10633C007474696E6773206F6E2052580A00416244
:10634C006F727465642065646974730A00696E7693
:10635C00616C69642073656C656374696F6E000DA4
:10636C000A496E76616C696420696E707574202DB3
:10637C0020646973636172646564210700536574FA
:10638C0074696E677320736176656420746F204541
:10639C004550524F4D0A0052657665727465642003
:1063AC0073657474696E67732066726F6D204545F2
:1063BC0050524F4D0A004C6F6164656420666163F6
:1063CC00746F72792064656661756C74730A004B26
:1063DC00657920616E64206368616E6E656C7320F4
:1063EC0072616E646F6D697A65640A004F70656ED8
:1063FC004C52536E67205458207374617274696EDA
:10640C00672000206F6E20485720006D6F64756CFC
:10641C0065206C6F636B65643F00342B340038006F
:10642C00382B340031320031322B340031360050ED
:10643C00504D0052535349005344410053434C00B8
:10644C00525844005458440041494E004C42454572
:10645C00500053504B54524D00534255530053551A
:10646C004D44004C4C494E440000070B0C101115C8
:10647C0000B6012A032E033003340337033C03B662
:10648C00013F03430348034C035003540358035C7C
:10649C0003620369036E0373038C028C028C028CFF
:1064AC0002160A1322312900000000022C072AA828
:0864BC002BD52BBA2BF72B00A6
:107E00000F92CDB7DEB7112484B714BE81FFF1D035
:107E100082E08093C00088E18093C10086E0809377
:107E2000C20080E18093C4008EE0CDD088249924E4
:107E3000CC24C394F5E0DF2EE1E1EE2E73E0F72EC3
:107E4000B6D0082F813479F4B2D08983C2D0898129
:107E5000823811F481E005C0813811F485E001C059
:107E600083E09ED09AC0823411F484E103C085344B
:107E700019F485E0B6D091C0853561F498D0082F0B
:107E800010E095D090E0982E8824802A912A880CC2
:107E9000991C82C0863521F484E0A3D080E0E1CF34
:107EA000843609F04CC083D082D0A82E80D0B82E62
:107EB00000E011E07CD0F80181938F01AE16D1F77C
:107EC00088D0FB2DF53489F4E0E0F1E00BC0F9999E
:107ED000FECF92BC81BC0894811C911C819180BD15
:107EE000FA9AF99AEA1598F358C08B2D863409F05E
:107EF00054C0F401F7BEE89507B600FCFDCFF401CD
:107F0000A0E0B1E02C9130E011968C91119790E0B7
:107F1000982F8827822B932B12960C01C7BEE895C9
:107F20001124329681E0A038B80761F7F401D7BE7A
:107F3000E89507B600FCFDCFE7BEE8952EC0843774
:107F4000F1F435D034D0182F32D0B82E42D0FB2DDA
:107F5000F63421F4F40105914F010CC0FB2DF534EA
:107F600049F4F999FECF92BC81BC0894811C911C04
:107F7000F89A00B5802F14D0115049F70EC08537FC
:107F800039F427D08EE10CD085E90AD08FE069CF93
:107F9000813511F488E017D01CD080E101D050CF9A
:107FA0009091C00095FFFCCF8093C600089580910A
:107FB000C00087FFFCCF8091C00084FD01C0A89560
:107FC0008091C6000895E0E6F0E098E19083808318
:107FD0000895EDDF803219F088E0F5DFFFCF84E10E
:107FE000DFCF1F93182FE3DF1150E9F7F2DF1F9166
:0E7FF0000895282E80E0E7DFEE27FF27099492
:027FFE0001057B
:0400000300007E007B
:00000001FF
